:020000040000FA
:1000000001308A000030A500831686008500831227
:1000100033200E201B202720642009281030840064
:100020001030A4002408250767208000840AA40B50
:100030001228A50A080080303C200830A3001F3099
:100040008400000848208403A30B21280800C03046
:100050003C200830A30017308400000848208403A7
:10006000A30B2D28080038303C2001303C20033001
:100070003C200F303C2008008600542004308500CE
:10008000542000308500542004308500542008009E
:10009000860054200630850054200230850054200C
:1000A00006308500542008000A30A200A100A10BF0
:1000B0005728A20B56280800FA30A200A100A10B75
:1000C0005F28A20B5E2808005C205C2008008200EC
:100200002034453444345534503449344334203454
:10021000313436344634383434342E342E34313498
:100220004B3420344D3445344D344F3452344934FA
:100230004134203446344C344134533448342E3421
:100240002E34363434342034423459345434453422
:1002500053342034443445342034523441344D3402
:100260002E342E3436343834203442345934543415
:1002700045345334203444344534203445344534F3
:10028000503452344F344D342E342E34503455348F
:100290004534523454344F34533420345034413480
:1002A0005234413420344C344334443420345934AF
:1002B00020345434453443344C34413444344F3482
:1002C0002E342E34523445344C3445345634413473
:1002D00044344F345234203444344534203431349F
:1002E0003234373476342E3420343134203461348F
:1002F0006D3470342E342E34383420344C3445343C
:10030000443453342E342E34343420344D34493470
:10031000433452344F3453345734493454344334CF
:100320004834453453342E342E34503452344F3400
:100330004734523441344D34413444344F345234D0
:100340002034443445344C3420343134363446344B
:1003500038343434203449344E34543445344734FA
:100360005234413444344F342E342E3449344E34D4
:1003700043344C34553459344534203453344F3499
:1003800046345434573441345234453420344D3497
:1003900050344C3441344234203443344F344E349E
:1003A000203445344E34533441344D3442344C348B
:1003B000413444344F3452342C342034533449348F
:1003C0004D3455344C34413444344F345234203459
:1003D00059342034503452344F3447345234413439
:1003E0004D34413444344F3452342E342E342E3470
:1003F0002E342E342E342E342E342E342E342E34ED
:02400E00F13F80
:00000001FF
